:100000000C948F000C94AE000C94AE000C94B803CA
:100010000C94AE000C94AE000C94AE000C94AE00A8
:100020000C94AE000C94AE000C94AE000C94AE0098
:100030000C94AE000C94AE000C94AE000C948D1F8A
:100040000C94AE000C94AE000C94AE000C94AE0078
:100050000C94AE000C94AE000C94AE000C94AE0068
:100060000C94AE000C94AE000C94AE000C94AE0058
:100070000C94AE000C94AE000C94AE000C94AE0048
:100080000C94AE000C9456080C94AE00920E0E0F19
:100090000E0F0E0FA20EB60EBD0EC60ED30E0E0F15
:1000A000E10EE80EDC0EEE0E0E0F0E0F0E0F2C0FF3
:1000B0000E0F0E0F0E0F0E0F0E0F0E0F0E0FF90E6E
:1000C000000F0E0F0E0F0E0F9A0E0E0F0E0F0E0FCB
:1000D0000E0F0E0F0E0F0E0F0E0F0E0F0E0F0E0F38
:1000E0000E0F0E0F070FA311AF11BB11C711D311C4
:1000F000DF11EC110412121220122E123C124A12BD
:100100005A1281128D129912A512B112BD12CA1281
:10011000E212F012FE120C131A13281338131124D2
:100120001FBEC0E0D0E1DEBFCDBF11E0A0E0B1E076
:10013000E4E2F4E400E00BBF02C007900D92A03EA1
:10014000B107D9F727E0A0EEB1E001C01D92A03CB5
:10015000B207E1F70E9490150C9410220C94000055
:10016000E199FECF21E0280F2EBB01969FBB6DBB0E
:10017000E29AE19A0895E199FECF21E0280F2EBB83
:1001800001969FBBE09A8DB30895E199FECF1EBA08
:100190001FBA8FEF8DBBE29AE19A0895E199FECFE5
:1001A0001EBA1FBA1DBAE29AE19A0895CF93DF935F
:1001B000C4EAD2E081E0888319821A828B83E091BD
:1001C000AC02F091AD0281818F5F8C83E091AE0231
:1001D000F091AF029181890F8D831E8268E0CE017C
:1001E0000E94E11F8F83DF91CF910895CF93DF931A
:1001F00080E490E00E94EF209093AD028093AC02E7
:1002000080E090E0E091AC02F091AD028034910585
:1002100029F0E80FF91F10820196F4CF81E0808366
:10022000E091AC02F091AD0288E08183E091AC02F4
:10023000F091AD0289E1828313821482158284ECED
:10024000868389E4878390E5908792E3918782870C
:1002500081ED8387A6E7B1E08CE090E02D91E091FD
:10026000AC02F091AD02E80FF91F208301968D31A9
:100270009105A1F7E091AC02F091AD0289EC858F78
:10028000A8E8B1E08EE190E02D91E091AC02F09110
:10029000AD02E80FF91F2083019687329105A1F77F
:1002A000E091AC02F091AD0288EC87A3A2E9B1E045
:1002B00088E290E02D91E091AC02F091AD02E80F60
:1002C000F91F2083019680339105A1F7E091AC02DC
:1002D000F091AD0287EC80ABABE9B1E081E390E057
:1002E0002D91E091AC02F091AD02E80FF91F20834F
:1002F000019688339105A1F7C091AC02D091AD026F
:1003000081EC88AF60E4CE010E94E11F8FAFDF91E6
:10031000CF910895CF93DF9388E390E00E94EF2080
:100320009093AF028093AE0280E090E0E091AE0245
:10033000F091AF028833910529F0E80FF91F108280
:100340000196F4CF81E08083E091AE02F091AF029C
:1003500087E08183E091AE02F091AF0289E1828370
:1003600084EC838389E4848390E5958392E3968388
:1003700087838EEC8087A3EAB1E089E090E02D913D
:10038000E091AE02F091AF02E80FF91F20830196D1
:1003900087319105A1F7E091AE02F091AF0285ECB3
:1003A000878BACE8B1E0ED0188E190E02991E09124
:1003B000AE02F091AF02E80FF91F208301968D3154
:1003C0009105A1F7E091AE02F091AF0282EC858F2A
:1003D00086E7868F81E3878F85EC80A381E290E0BA
:1003E0002D91E091AE02F091AF02E80FF91F20834A
:1003F000019686329105A1F7E091AE02F091AF022D
:1004000080EC86A387EC87A3ABE9B1E088E290E0BB
:100410002D91E091AE02F091AF02E80FF91F208319
:1004200001968F329105A1F7C091AE02D091AF0233
:1004300081EC8FA768E3CE010E94E11F8FABDF91B3
:10044000CF910895CF93DF93C2EBD2E080EC888305
:1004500082E8898386E08A831B821C828AE58D83F9
:1004600081E38E831F8286E18887198684E18A87EB
:1004700066E087EB92E00E94E11F8B8365E0CE018E
:100480000E94E11F8C83DF91CF9108950F931F93FA
:10049000CF93DF93CDB7DEB7A8970FB6F894DEBF42
:1004A0000FBECDBF85E390E00E94EF20FC0190934A
:1004B000B1028093B00280EC808382E0818380E38C
:1004C0008283138214828AE5858381E3868317827F
:1004D00089E180871186128680E8838785E084879A
:1004E00080EE8A8F8FEF8B8F8C8F94EE9D8F8E8F07
:1004F0008F8F95EE98A389A38AA396EE9BA38CA3D6
:100500008DA397EE9EA38FA388A7FE017A968DE018
:1005100090E0A091B002B091B102A80FB91F208164
:100520002C93A091B002B091B102A80FB91F218104
:1005300011962C93A091B002B091B102A80FB91FEF
:10054000228112962C93039633968C31910509F7EC
:10055000198231E53A831B821C822CEF2D8341E006
:100560004E833F8340E1488719862A8752E05B87A4
:100570003C874D871E862F8753E0588B398B4A8BDB
:100580001B8A2C8B54E05D8B3E8B4F8B188E298FF2
:10059000FE013196A091B002B091B102A80FB91F2F
:1005A00020812C93A091B002B091B102A80FB91F85
:1005B000218111962C93A091B002B091B102A80FA5
:1005C000B91F228112962C93A091B002B091B10272
:1005D000A80FB91F238113962C93A091B002B0915C
:1005E000B102A80FB91F248114962C930596359655
:1005F0008533910579F60091B0021091B102F801AE
:100600006281C80105960E94E11FF8018383009171
:10061000B0021091B10265E0C8010E94E11FF8012B
:100620008483A8960FB6F894DEBF0FBECDBFDF91CE
:10063000CF911F910F9108958091AC029091AD02DE
:100640000E9487218091AE029091AF020E94872183
:100650008091B0029091B1020C948721EF92FF92A9
:100660000F931F93CF93DF930E94F6000E948A019D
:100670000E9446020E9422020E94D6001FB7F894F0
:1006800084EAE82E82E0F82EC0E0D0E0F701619124
:100690007F01CE010E94B0002196C830D105B1F78C
:1006A000C0E0D0E0FC2EF8E0FF0EE091AC02F0914B
:1006B000AD02818128E0829FC0011124C817D907AB
:1006C0004CF4EC0FFD1F60818F2D90E00E94B00074
:1006D0002196E8CFC0E0D0E00C2F0F0DE091AE02E4
:1006E000F091AF02818128E0829FC0011124C817D8
:1006F000D9074CF4EC0FFD1F6081802F90E00E9421
:10070000B0002196E9CFC0E0D0E08C2F800FE091BF
:10071000B002F091B102228130E02C5F3F4F2C17E4
:100720003D0744F0EC0FFD1F608190E00E94B00097
:100730002196EBCFC2EBD2E02091B40230E02C5FE7
:100740003F4FAE01425B52402417350744F0699198
:1007500001E0080F90E00E94B000802FEDCF1FBF96
:10076000DF91CF911F910F91FF90EF900C941C039C
:100770001F920F920FB60F9211240BB60F922F9368
:100780003F934F935F936F937F938F939F93AF9319
:10079000BF93EF93FF931092E10180E00E94FA1E55
:1007A000FF91EF91BF91AF919F918F917F916F9149
:1007B0005F914F913F912F910F900BBE0F900FBE05
:1007C0000F901F901895CF93DF931F92CDB7DEB790
:1007D000898321E0AE014F5F5F4F60E080E00E94BF
:1007E000D90F8093E0010F90DF91CF91089580B3EE
:1007F00082FB882780F9089580916A008061809348
:100800006A0080916A008F7D80936A0089B7846056
:1008100089BF60E080E00E94E81E0E94F70381111A
:1008200005C061E00E94E81E80E005C062E080E053
:100830000E94E81E81E00C94E303CF938091E101D4
:100840008F5F8093E1018730D0F10E94F703C82FBA
:1008500080E00E94041F811104C08091E001882380
:1008600061F180910601C81731F180E0C11111C01A
:100870000E94F11E682F6D7F80E00E94E81E80E0DC
:100880000E94F11E682F616080E00E94E81E80E0F7
:1008900010C00E94F11E682F6E7F80E00E94E81E4B
:1008A00080E00E94F11E682F626080E00E94E81ED6
:1008B00081E00E94E303C09306011092E001CF9112
:1008C00008950C94C5008091BF02882329F01092EE
:1008D000BF020E94CE00FFCF0895CF93DF93982FE1
:1008E000EB01FA01D901813309F451C028F48E32A9
:1008F000B1F08F3211F168C0833309F463C008F49A
:100900005FC0843309F060C08091C0028083809111
:10091000BD0281838091BE02828383E00CC010827D
:1009200088E2818388E18283138214828CE085834C
:1009300081E0868387E08C933FC0898181113EC02E
:100940009A819230A1F060F4992369F09130E1F539
:1009500090839183128213821482158296E015C0CF
:10096000953070F131C094E2908391E00EC0C2EBFB
:10097000D1E090E0983018F42881208301C01082E3
:100980009F5F219631969C30A9F79C931EC0898168
:10099000811118C08091BD028038B9F08A81813000
:1009A00059F0823089F481E08093BF0280E880931F
:1009B000BD029093C00209C080E007C082E805C074
:1009C00083E803C081E801C08CECDF91CF910895EA
:1009D000D098D298D39AD49AD59AB89ABB98BA9804
:1009E000B998BD9ABE9ABF9AA29AA39AA498A598BC
:1009F000A69AA79A8A9812981398E1E6F0E0808167
:100A00008E7F8083A4E6B0E08C9181608C938C9182
:100A100082608C938C9184608C938C91877F8C9373
:100A2000A09AA19AA29AA498A39AA598808182607C
:100A30008083808184608083808188608083169A2F
:100A4000149A159A179A089581E08093E301089506
:100A5000AF9AAE9A80E00E94F11E682F677E80E018
:100A60000E94E81E80E00895AF98AE9880E00E9452
:100A7000F11E682F606180E00E94E81E80E008950A
:100A80000E94E70C9091E201882399F1911113C023
:100A900080E00E942106833870F080E00E94F11E01
:100AA000682F6B7F80E00E94E81E81E08093E20166
:100AB0000E9428050BC08091E201813039F480E06A
:100AC0000E942106813410F41092E2018091E3012A
:100AD0001092E301882371F10E94340580E00E94A6
:100AE000F11E682F646080E00E94E81E82E00C9492
:100AF000E30391110EC080E00E942106833848F084
:100B00000E94F703811105C081E08093E2010C94FB
:100B100028058091E201813069F480E00E9421067D
:100B2000803420F41092E2010C9434050E94F70303
:100B30008130C1F30895823059F4AF98AE98A895EA
:100B400084EF91E00E94541FAF9AAE9A80E008951E
:100B50008FEF089584E008950F931F93CF93DF9351
:100B60001F92CDB7DEB78E010F5F1F4F21E040E02F
:100B700060E070E00E94E20B89810F90DF91CF91DD
:100B80001F910F9108950F931F93CF93DF931F929F
:100B9000CDB7DEB769838E010F5F1F4F21E040E0C4
:100BA00060E070E00E944A0B0F90DF91CF911F919F
:100BB0000F910895CF93DF93D82FC62F0E94AC05D5
:100BC000C15061E070E001C0660FCA95EAF7609518
:100BD00068238D2FDF91CF910C94C305CF93DF93C2
:100BE000D82FC62F0E94AC05C15061E070E001C053
:100BF000660FCA95EAF7682B8D2FDF91CF910C9481
:100C0000C30596B1987F892B86B9089527B12F73B4
:100C100030E4839FC0011124822B87B90895379A4D
:100C200085E00E94010680E00E9406063D9A089534
:100C300097B1907E8F71892B87B90895349A369A2F
:100C400008950E9418060E941E06349BFECF85B1AF
:100C50000895CF93DF9385E090E00E94BB0028E0E9
:100C6000829FC00111240097D1F0EC01CE010196C2
:100C70000E94BB009E012E5F3F4F87FD08C0C90147
:100C80000E94BB0090E00596C80FD91FEFCFC901A5
:100C90000E94BB0090E005968C0F9D1F22C084E04F
:100CA00090E00E94BB0038E0839FE0011124209770
:100CB00051F483E090E00E94BB0098E0899FE0013E
:100CC0001124209761F0CE0101960E94BB009E0185
:100CD00048E0849F200D311D1124C90102C080E02D
:100CE00090E0DF91CF910895CF93DF93811108C0F9
:100CF000EB010E942906888399831A8283E001C050
:100D00008FEFDF91CF910895CF92DF92EF92FF9214
:100D10000F931F93CF934D33F8F4F901C42FDB01E8
:100D2000ED90FC904083811107C089010F5F1F4F38
:100D30006701C40ED11C03C081E08C0F0EC0EC14FF
:100D4000FD04D1F3C7010E94BB00F80181938F011C
:100D5000FFEFEF1AFF0AF3CF8FEFCF911F910F91A3
:100D6000FF90EF90DF90CF900895CF92DF92EF92B7
:100D7000FF920F931F93CF93DF93FC01C080D1802C
:100D8000842F90E09C012C0D3D1D21303840B8F49B
:100D9000C42FDFB7F8948B017B01E80EF91E0E1506
:100DA0001F0551F0F80161918F01C6010E94B0004A
:100DB000FFEFCF1ADF0AF3CFDFBF8C2F01C08FEF19
:100DC000DF91CF911F910F91FF90EF90DF90CF9027
:100DD0000895E82FF0E0E851FE4F6083613011F490
:100DE0000C940A20611102C00C940C2008959F926B
:100DF000AF92BF92CF92DF92EF92FF920F931F9329
:100E0000CF93DF93F82E8B0185E090E00E94BB002A
:100E100028E0829FC0011124009711F480E061C096
:100E2000EC01CE0101960E94BB00AE01485F5F4F0E
:100E30006A0187FF06C0C6010E94BB00893171F7B5
:100E40000EC0CA010E94BB008931A9F3CE010296EF
:100E50000E94BB0090E00596C80FD91FE2CFCE01DB
:100E60000A960E94BB0050E1859FC00DD11D112440
:100E7000CE010C960E94BB00F81680F6CF2CD12C28
:100E800065E0F69E90011124F90143E0849FE00D96
:100E9000F11D1124CE0FDF1FCE010D960E94BB0065
:100EA000982ECE010E960E94BB00A82ECE010F9662
:100EB0000E94BB00B82ECE0140960E94BB00E82ED7
:100EC000CE0141960E94BB00F910A8CFF801A08284
:100ED000B182E282F601E851FE4F8081F8018383FE
:100EE00084E0DF91CF911F910F91FF90EF90DF9001
:100EF000CF90BF90AF909F900895CF93DF93C82F6E
:100F0000D62F613019F40E940A2004C0611109C073
:100F10000E940C20811105C0EC2FF0E0E851FE4F3B
:100F2000D08380E0DF91CF91089580E00895FC01A7
:100F300084E180831182128283E00895982F827069
:100F400091FF06C0669561706093E60180E00895A8
:100F500090FF04C061706093E70108958FEF0895DA
:100F60008091E601880F82709091E701892B809330
:100F7000C1020895813031F48091E5018F5F809343
:100F8000E50107C08091E401811103C081E08093F5
:100F9000E40180E0089580E090E00E94BB008F3F74
:100FA00011F40C942E030895BC01809171008E7F82
:100FB00080937100809171008D7F8093710080E932
:100FC00091E00E94D220862F603138F07727CB0144
:100FD000409797FD019695958795809370000895A9
:100FE000909A919A1092FC011092FB0184E190E09A
:100FF0000E94D407E4E7F0E080818460808310924F
:1010000097028081816080838081806480830895DD
:101010008E7F91E0611101C090E0982B9093720057
:1010200008959093FC018093FB010895E4E7F0E0BC
:1010300080818F70806A80830895E4E7F0E080818A
:101040008F70806D8083089580937300E4E7F0E0F3
:1010500080818F70806880830895882329F0809133
:1010600074008F70806C04C0809174008F708068F1
:10107000809374000895909197029111FCCF92E0B3
:10108000909397028E7F80939602942FABE4B2E008
:10109000FA018E2F891B861718F481918D93F9CF51
:1010A00010924A02609349020C9416081F920F9204
:1010B0000FB60F9211240BB60F922F933F934F93BD
:1010C0005F936F937F938F939F93AF93BF93EF93B0
:1010D000FF9380917100887F803709F467C020F505
:1010E000803209F44AC080F4883009F443C038F4EF
:1010F0008111BDC0809174008F70806DB4C080314B
:10110000C9F18831D1F1B3C0883309F44AC028F459
:10111000883299F1803389F1AAC0803609F446C03B
:10112000883609F443C0A3C0803A09F45CC080F457
:10113000883809F454C030F48837C1F1803809F494
:1011400040C095C08039E9F1883909F448C08FC0A2
:10115000883B09F466C038F4883A09F456C0803BED
:1011600009F453C084C0803C09F479C0883C09F478
:1011700076C07DC0809196020EC0E0914A028091B7
:101180004902E81758F481E08E0F80934A02F0E09C
:10119000E55BFD4F80810E94240869C00E941D0804
:1011A00064C0809174008F7080685DC085E080931A
:1011B000970281E08093FD01809173008093FE018E
:1011C00042C0E091FD0181E08E0F8093FD0190917E
:1011D0007300F0E0E250FE4F90838032A0F180E097
:1011E0000E942D0844C0809174008F70806C8093A1
:1011F0007400E091FB01F091FC013097B1F16EEFCA
:1012000071E08091FD01099530C084E080939702E0
:10121000E091F901F091FA016EEF71E08091FD012A
:101220000995E0914A0281E08E0F80934A02F0E036
:10123000E55BFD4F80818093730090914A0280911D
:101240004902981728F4809174008F70806C04C054
:10125000809174008F7080688093740008C08091C2
:1012600074008F70806C8093740010929702FF91CD
:10127000EF91BF91AF919F918F917F916F915F910E
:101280004F913F912F910F900BBE0F900FBE0F907B
:101290001F90189527E030E090E0AC01022E02C0CC
:1012A000559547950A94E2F740FF02C08D9801C01A
:1012B0008D9A000000000000000000000000000007
:1012C000000000000000000000000000000000001E
:1012D000000000000000000000000000000000000E
:1012E00000000000000000000000000000000000FE
:1012F00000000000000000000000000000000000EE
:1013000000008C98000000000000000000000000B9
:1013100000000000000000000000000000000000CD
:1013200000000000000000000000000000000000BD
:1013300000000000000000000000000000000000AD
:10134000000000000000000000000000000000009D
:10135000000000008C9A2150310908F09ECF8D9832
:10136000000000000000000000000000000000007D
:10137000000000000000000000000000000000006D
:10138000000000000000000000000000000000005D
:10139000000000000000000000000000000000004D
:1013A000000000000000000000000000000000003D
:1013B0008C9880B3000000000000000000000000D6
:1013C000000000000000000000000000000000001D
:1013D000000000000000000000000000000000000D
:1013E00000000000000000000000000000000000FD
:1013F00000000000000000000000000000000000ED
:10140000000000008C9A00000000000000000000B6
:1014100000000000000000000000000000000000CC
:1014200000000000000000000000000000000000BC
:1014300000000000000000000000000000000000AC
:10144000000000000000000000000000000000009C
:1014500000000000000085FB882780F991E08927C3
:101460000895AC018D9828E030E080E00000000095
:10147000000000000000000000000000000000006C
:10148000000000000000000000000000000000005C
:10149000000000000000000000000000000000004C
:1014A000000000000000000000000000000000003C
:1014B0000000000000000000000000008C98880F71
:1014C000859981600000000000000000000000001D
:1014D000000000000000000000000000000000000C
:1014E00000000000000000000000000000000000FC
:1014F00000000000000000000000000000000000EC
:1015000000000000000000000000000000000000DB
:10151000000000008C9A2150310909F0A7CF8D9A64
:10152000452B11F08D9801C08D9A0000000000003D
:1015300000000000000000000000000000000000AB
:10154000000000000000000000000000000000009B
:10155000000000000000000000000000000000008B
:10156000000000000000000000000000000000007B
:10157000000000000000000000008C980000000047
:10158000000000000000000000000000000000005B
:10159000000000000000000000000000000000004B
:1015A000000000000000000000000000000000003B
:1015B000000000000000000000000000000000002B
:1015C0000000000000000000000000008C9A8D98D0
:1015D0000895959894988D988C98000000000000CC
:1015E00000000000000000000000000000000000FB
:1015F00000000000000000000000000000000000EB
:1016000000000000000000000000000000000000DA
:1016100000000000000000000000000000000000CA
:10162000000000000000000000008C980000000096
:1016300000000000000000000000000000000000AA
:101640008D98000000000000000000000000000075
:10165000000000000000000000000000000000008A
:10166000000000000000000000000000000000007A
:10167000000000000000000000000000000000006A
:10168000000000000000000000000000000000005A
:1016900000000895DF92EF92FF920F931F93CF9374
:1016A000DF93F62EE72ED42FC22FDFB6F8948D9A53
:1016B000000000000000000000000000000000002A
:1016C000000000008C9A880F0E944A09D23041F431
:1016D0008E2D0E944A098F2D0E944A09780103C06D
:1016E000D130E1F7F8CFCC2339F0F70181917F01B8
:1016F0000E944A09C150F7CF8D9A000000000000F7
:1017000000000000000000000000000000000000D9
:1017100000000000000000000000000000000000C9
:1017200000000000000000000000000000000000B9
:1017300000000000000000000000000000000000A9
:10174000000000000000000000008C980000000075
:101750000000000000000000000000000000000089
:101760008D98000000000000000000000000000054
:101770000000000000000000000000000000000069
:101780000000000000000000000000000000000059
:101790000000000000000000000000000000000049
:1017A0000000000000000000000000000000000039
:1017B0000000DFBEDF91CF911F910F91FF90EF905E
:1017C000DF900895AF92BF92DF92EF92FF920F9356
:1017D0001F93CF93DF93E62EB72EF42EC22FD82F70
:1017E000DD0FDFB6F8948D9A0000000000000000C5
:1017F0000000000000000000000000008C9A82E061
:10180000481305C08D2F0E944A098B2D04C0E1E0CA
:101810004E1306C08D2F0E944A098E2D0E944A0940
:1018200000000000000000000000000000000000B8
:1018300000000000000000000000000000000000A8
:101840000000000000000000000000000000000098
:101850000000000000000000000000000000000088
:101860000000000000000000000000000000000078
:10187000FF2069F08C988D9A0000000000000000A5
:101880000000000000000000000000008C9A8D2F76
:1018900081600E944A0978010C2F10E0C0E0D0E07E
:1018A0005801F1E0AF1AB1080C171D0771F081E083
:1018B00090E0AC16BD0611F080E090E00E94310A85
:1018C000F70181937F012196EFCF8D9A00000000F0
:1018D0000000000000000000000000000000000008
:1018E00000000000000000000000000000000000F8
:1018F00000000000000000000000000000000000E8
:1019000000000000000000000000000000000000D7
:101910000000000000000000000000008C980000A3
:1019200000000000000000000000000000000000B7
:1019300000008D9800000000000000000000000082
:101940000000000000000000000000000000000097
:101950000000000000000000000000000000000087
:101960000000000000000000000000000000000077
:101970000000000000000000000000000000000067
:1019800000000000DFBEDF91CF911F910F91FF900B
:10199000EF90DF90BF90AF9008959091BA05986056
:1019A0009093BA0590FD12C0262FAEEFB5E0FB0173
:1019B0009E2F921B981718F491919D93F9CF8093C5
:1019C00049068091BA0581608093BA050895809197
:1019D000980208958093F0066093EF068F3F19F404
:1019E00010929902089581E0809399020895EBEB9B
:1019F000F5E0108280E8818381E08283838381E542
:101A0000848389E2858380E68683178210868187B6
:101A100087E782878BE008950F931F93CF93DF931F
:101A2000CDB7DEB7CC54D1090FB6F894DEBF0FBEE8
:101A3000CDBF082F8091FC0589838091F10690E04D
:101A40000196880F991F880F991F9091F206937045
:101A5000892B8A8362E0CE0101960E94E11F8B836D
:101A600080919E068C8380913707880F880F8D8325
:101A70008091F3068E830F838091F1068C3219F4E6
:101A8000188618E001C017E0011113C080919D066F
:101A9000882379F0EBEBF5E0810F181751F0919165
:101AA000A1E0B0E0AC0FBD1FA10FB11D9C931F5F63
:101AB000F4CF612FCE0101960E94E11FE1E0F0E03A
:101AC000EC0FFD1FE10FF11D8083AE014E5F5F4FF4
:101AD000612F8091FC050E943B088091BA058E7FA2
:101AE0008093BA05C45BDF4F0FB6F894DEBF0FBE1C
:101AF000CDBFDF91CF911F910F910895AF92CF92FB
:101B0000EF92FF920F931F93CF93DF931F92CDB766
:101B1000DEB710929D0620919A02422F50E09091DC
:101B2000F106FA01E45BF94F90838091F306FA0124
:101B3000E156F94F80832F5F2F3418F420939A02D7
:101B400002C010929A029A3009F4ACC028F4943082
:101B500099F0963059F080C19E3209F468C19033F3
:101B600009F4E6C09C3209F077C1D1C0813009F098
:101B700073C10E94F70CDAC0813281F160F48130C8
:101B800031F1F0F0803209F067C160E08BEB95E055
:101B90000E94311DCBC0863209F45BC020F4823232
:101BA00009F46AC059C1873209F446C08D3209F080
:101BB00053C16BEB75E08091F6060E94A81E42C0EF
:101BC0006091F7068091F6060E94EA0CB1C0809100
:101BD000F0068093BB058091EF0660C06091FA0625
:101BE000662321F180919B0290919C022091F60640
:101BF00030E0AC0155272417350709F02BC120919F
:101C0000F70630E0892F99272817390709F022C1F4
:101C10002BEB35E04091FB0688EF96E00E943C1DDF
:101C200080939D068F3F09F083C018C12BEB35E0F0
:101C30004091FB0660E0F0CF6BEB75E08091F6061B
:101C40000E94881D80939D068F3F09F071C08DEC26
:101C500006C1A090FD06C090FC06E090FB06009136
:101C6000FA062091F9064091F8066091F7068091F6
:101C7000F6060E940A1EE6CF80919B0290919C027C
:101C8000019611F481E090E090939C0280939B0276
:101C900090919B0280919C029093BB058093BC0520
:101CA00082E044C0813181F08231C9F0803109F095
:101CB000D3C06BEB75E08091F6060E9474068093AA
:101CC0009D068F3FA9F5C8C02BEB35E04091F90682
:101CD00067EF76E08091F6060E948406A1CF80919E
:101CE000F60681110DC04091F406435069EF76E08D
:101CF00087EF96E00E94B50680939D0680E001C0C4
:101D000081EC90919D069F3F09F0A9C0A7C0482F84
:101D100050E04D32510508F081C0FA01EA5BFF4FF7
:101D20000C94E6208BEB95E00E94970780939D062C
:101D300080E095C081E080939D060E94AA05809373
:101D4000BB05F6CF9091F7068091F806913019F413
:101D5000843009F481C0843019F40E942405E8CF4E
:101D60000E949B058F3F21F78CEC79C06BEB75E0EF
:101D70008091F7060E946211D9CF4BEB55E060913C
:101D8000F8068091F7060E946D110AC02091FA06AC
:101D90004091F9066091F8068091F7060E94B2140E
:101DA00080939D06DFCF4BEB55E06091F806809164
:101DB000F7060E942B11F4CF8091F8060E94BA0713
:101DC000D1CF6091F9068091F8060E949E07CACF94
:101DD0000E94B0078093BB0581E0A8CF8091F806F0
:101DE00081113CC06BEB75E08091F7060E94DB1E11
:101DF00017CF6091FB068091F7060E947D0796CF72
:101E00006BEB75E08091F7060E94F7068FCF60912B
:101E1000F9068091F7060E94950788CF2DE936E0F4
:101E20004BEB55E066EF76E00E946D0418C0209100
:101E3000F4062350AE014F5F5F4F7A010BEB15E0C4
:101E400049EF56E066EF76E00E94132080939D06EE
:101E5000898105C085EC03C081EC01C089EC0E943A
:101E60000C0D0F90DF91CF911F910F91FF90EF908C
:101E7000CF90AF9008958091BA0580FF99C04091AE
:101E8000000662E08EEF95E00E94EE1F811190C087
:101E900060914906E62FF0E0E350FA4F615040812F
:101EA0008EEF95E00E94EE1F811182C08091FE05A9
:101EB00080939E068091FF05869586958093F10616
:101EC000209101062093FC0590910206392F36954A
:101ED00036953093370793709093F20690910306EE
:101EE0009093F30680FF3FC08091F006281360C0F6
:101EF0008091BA058E7F8093BA0510929C0610924D
:101F0000380780910406882321F080919D02833058
:101F100030F181E02CE490919E028917D0F4482F93
:101F200050E0BA0161507109269FD001279FB00D82
:101F30001124AE53BD4F249FF001259FF00D1124B5
:101F4000EE53FD4F922F01900D929A95E1F78F5F1E
:101F5000E2CF915090939E0210929D0208958F5F60
:101F600080939D020895809149068830D8F090E0D2
:101F70009C01275031093093F5062093F40646E082
:101F80000197EAEFE40F242F30E02817390774F4A3
:101F9000F0E0EF50F94FD901A250BA4F2C912583B0
:101FA0004F5FEFCF1092F5061092F4060C947E0D61
:101FB0000895CF92DF92EF92FF920F931F93CF93EA
:101FC000DF93C0919E02CA3008F05EC0022F7A01F2
:101FD000D62EC82E90914B069F5F90934B061CE423
:101FE0001C9FE0011124CE53DD4F990F990F9C8364
:101FF00082E08D8384E08E838C2D0E940E1F8F8360
:10200000C0919E021C9FE0011124CE53DD4FC88673
:102010008C2D0E94171F8F77D82AD98680919E0217
:10202000282F30E0002319F0F701908101C09FEFC5
:102030004CE4429FF001439FF00D1124EE53FD4FFD
:102040009287023018F0F701918101C09FEF4CE4B4
:10205000429FF001439FF00D1124EE53FD4F9387F3
:10206000033018F0F701928101C09FEF4CE4429FCA
:10207000F001439FF00D1124EE53FD4F94878F5FC5
:1020800080939E0280E001C081E0DF91CF911F919B
:102090000F91FF90EF90DF90CF900895CF93DF9353
:1020A00081E080933807C2ECD2E08091F00688830B
:1020B0008091EF0683708061898380914A068B83CB
:1020C00062E0CE010E94E11F8A836DE0CE010E9492
:1020D000E11F8D8743EC52E06DE08091F006DF91C7
:1020E000CF910C943B088091F0068F3F69F080916E
:1020F0009E02882349F080913807811105C08091A4
:10210000BA0580FF0C944E1008951F93CF93DF9370
:10211000BB98BA98B998B89AC09880B5846080BDC9
:1021200084E690E00E94401F26B323FB112710F99C
:1021300096B392FBDD27D0F986B381FBCC27C0F99B
:10214000C09A84E690E00E94401F86B383FB8827F4
:1021500080F9181302C0212F01C022E086B382FB50
:10216000882780F9D81302C09D2F01C092E086B362
:1021700086958170C81302C08C2F01C082E02111A6
:102180000EC0911104C08230D1F582E739C092307F
:10219000B1F5882351F1823091F586E731C02230C4
:1021A000B1F4911106C0882311F1823041F58AE71C
:1021B00027C0923031F48823E1F0813001F58EE7B9
:1021C0001FC08230C1F08130D1F482E819C0923052
:1021D00031F4823091F0813091F486E811C0913071
:1021E00071F4823061F488E80BC084E709C088E7A5
:1021F00007C08CE705C080E803C084E801C080E028
:1022000090B59B7F90BD811101C080E7DF91CF9198
:102210001F9108950E94F0070E94851080934A063E
:102220006FEF0E9408088DEC9CE00E9411088FEF70
:102230008093F00681E080934B061092EF06109297
:102240009C0680939802089580914A06811102C0ED
:102250000C9485100895DA0181112EC0633060F569
:102260008CE0689FF0011124E75CF84F84818C9327
:10227000808111968C931197828112968C9312977C
:10228000838113968C93139784818B7F8230B1F472
:10229000818114968C931497828115968C9315974F
:1022A000838116968C9316978481863049F48681B3
:1022B00017968C9388E008958FEF089584E0089531
:1022C00087E00895FB0197E09083811103C083E0CC
:1022D000818301C0118282E00895DA0181111AC060
:1022E0006330C0F48CE0689FF0011124E75CF84F84
:1022F00081E090E0038002C0880F991F0A94E2F702
:102300008C93838111968C931197838112968C9371
:1023100083E008958FEF0895DC0116968C9116974F
:102320001296EC9112974E2F50E0882309F461C069
:102330004730510508F0CDC0FA01ED58FF4F139614
:102340008C910C94E6204BB321E030E0B90102C03F
:10235000660F771F8A95E2F7CB01842B61C048B3E3
:1023600021E030E0B90102C0660F771F8A95E2F7DD
:10237000CB01842B63C045B321E030E0B90102C03A
:10238000660F771F8A95E2F7CB01842B65C042B3B5
:1023900021E030E0B90102C0660F771F8A95E2F7AD
:1023A000CB01842B67C043B121E030E0B90102C00A
:1023B000660F771F8A95E2F7CB01842B69C04091A5
:1023C000620021E030E0B90102C0660F771F8A95F4
:1023D000E2F7CB01842B6BC04091650021E030E037
:1023E000B90102C0660F771F8A95E2F7CB01842BF3
:1023F0006EC04730510508F06CC0FA01E658FF4F37
:1024000013968C910C94E6204BB321E030E0B90197
:1024100002C0660F771F8A95E2F7CB01809584236F
:102420008BBB089548B321E030E0B90102C0660FCC
:10243000771F8A95E2F7CB018095842388BB0895A6
:1024400045B321E030E0B90102C0660F771F8A95DD
:10245000E2F7CB018095842385BB089542B321E048
:1024600030E0B90102C0660F771F8A95E2F7CB0111
:102470008095842382BB089543B121E030E0B90107
:1024800002C0660F771F8A95E2F7CB0180958423FF
:1024900083B908954091620021E030E0B90102C0A3
:1024A000660F771F8A95E2F7CB018095842380938E
:1024B000620008954091650021E030E0B90102C05A
:1024C000660F771F8A95E2F7CB018095842380936E
:1024D00065000895DC0117968C9117971296EC9180
:1024E00012974E2F50E0882309F461C04730510500
:1024F00008F0CDC0FA01EF57FF4F13968C910C9462
:10250000E6204BB321E030E0B90102C0660F771F2F
:102510008A95E2F7CB01842B61C048B321E030E01B
:10252000B90102C0660F771F8A95E2F7CB01842BB1
:1025300063C045B321E030E0B90102C0660F771FE8
:102540008A95E2F7CB01842B65C042B321E030E0ED
:10255000B90102C0660F771F8A95E2F7CB01842B81
:1025600067C043B121E030E0B90102C0660F771FB8
:102570008A95E2F7CB01842B69C04091620021E08B
:1025800030E0B90102C0660F771F8A95E2F7CB01F0
:10259000842B6BC04091650021E030E0B90102C09E
:1025A000660F771F8A95E2F7CB01842B6EC0473008
:1025B000510508F06CC0FA01E857FF4F13968C9153
:1025C0000C94E6204BB321E030E0B90102C0660F65
:1025D000771F8A95E2F7CB01809584238BBB089502
:1025E00048B321E030E0B90102C0660F771F8A9539
:1025F000E2F7CB018095842388BB089545B321E0A1
:1026000030E0B90102C0660F771F8A95E2F7CB016F
:102610008095842385BB089542B321E030E0B90161
:1026200002C0660F771F8A95E2F7CB01809584235D
:1026300082BB089543B121E030E0B90102C0660FCA
:10264000771F8A95E2F7CB018095842383B908959B
:102650004091620021E030E0B90102C0660F771FAF
:102660008A95E2F7CB0180958423809362000895D8
:102670004091650021E030E0B90102C0660F771F8C
:102680008A95E2F7CB0180958423809365000895B5
:10269000EF92FF921F93CF93DF93CDB7DEB7E09712
:1026A0000FB6F894DEBF0FBECDBF28E1FE017996CC
:1026B000DF01922F1D929A95E9F791E09B8F37E009
:1026C0003C8F9D8F98A39BA335E03CA332E03DA3B4
:1026D0003FEF3EA398A79BA736E03CA733E03DA77A
:1026E00098ABDE01119601900D922A95E1F7E62E46
:1026F000F12CACE06A9FF0011124E75CF84F948163
:102700009B7F9230E1F1142F81112FC0F70183E0FC
:10271000EE0FFF1F8A95E1F781E090E08C0F9D1F7F
:10272000E80FF91F8081882319F0813069F01DC0FE
:102730004F3F21F4CF010E948C1117C0411115C0E9
:10274000CF010E946A1211C04F3F11F4868103C06D
:1027500041110BC087816381882321F081810E9410
:10276000EE0503C081810E94DA058CE08E9DF001A8
:102770008F9DF00D1124E75CF84F10831583E096D0
:102780000FB6F894DEBF0FBECDBFDF91CF911F9182
:10279000FF90EF900895CF92DF92EF92FF920F9308
:1027A0001F93CF93DF93CDB7DEB7E0970FB6F894C2
:1027B000DEBF0FBECDBF98E1FE017996DF01892F04
:1027C0001D928A95E9F781E08B8F27E02C8F8D8F02
:1027D00088A38BA325E02CA322E02DA32FEF2EA30B
:1027E00088A78BA726E02CA723E02DA788ABDE01C6
:1027F000119601900D929A95E1F7DE0111967D01F7
:1028000009E317E0D12CCC24C394F7014581D8010A
:102810004C9311964C93119712961C9212978481A7
:1028200013968C9313971496CC926D2D80E00E9492
:102830004813D394B8E0EB0EF11C045F1F4FE3E0A4
:10284000DE12E3CFE0960FB6F894DEBF0FBECDBF29
:10285000DF91CF911F910F91FF90EF90DF90CF907C
:102860000895EF92FF921F93CF93DF93CDB7DEB71A
:10287000E0970FB6F894DEBF0FBECDBF28E1FE0192
:102880007996DF01922F1D929A95E9F791E09B8F3F
:1028900037E03C8F9D8F98A39BA335E03CA332E0AB
:1028A0003DA33FEF3EA398A79BA736E03CA733E0AC
:1028B0003DA798ABDE01119601900D922A95E1F7A4
:1028C000E62EF12CACE06A9FF0011124E75CF84F92
:1028D00094819130D9F1142F81112FC0F70183E039
:1028E000EE0FFF1F8A95E1F781E090E08C0F9D1FAE
:1028F000E80FF91F8081882319F0813069F01DC02D
:102900004F3F21F4CF010E948C1117C0411115C017
:10291000CF010E946A1211C04F3F11F4868103C09B
:1029200041110BC087816381882321F081810E943E
:10293000EE0503C081810E94DA058CE08E9DF001D6
:102940008F9DF00D1124E75CF84F1583E0960FB6CC
:10295000F894DEBF0FBECDBFDF91CF911F91FF90E6
:10296000EF900895811145C0633008F042C0A62F52
:10297000B0E08CE0689FF0011124E75CF84F84819F
:102980008630B9F19FEF940F9A3F30F44183228350
:1029900082E08483238727C09E3F28F041831282F0
:1029A00082E0848321C04C3F39F481E084834081FC
:1029B00080E00E9448131BC04B3FD9F427FD19C08B
:1029C000813011F48CEF01C0818187838CE08A9F74
:1029D000F0018B9FF00D1124E75CF84F86E08483B3
:1029E0002683118610864FEF80E00E94311480E02C
:1029F00008958FEF08951F93CF93DF93C9E3D7E036
:102A000010E08C818630A9F4888599850196998794
:102A100088872E814AE0249F900111248217930712
:102A200008F11C822A814F81612F80E00E94B2143C
:102A300019C099818FEF890F8A3FA0F48B8582504E
:102A40008B8781110FC08D81882329F08F3F51F42E
:102A50009B8740E003C08A818B874FEF612F80E026
:102A60000E9431142C961F5F133059F6DF91CF91DD
:102A70001F9108950E9461040E94E8040E94CB0700
:102A80000E94E90A0E94CB130E940F060E94CF15F4
:102A90000E9452160E94201F88B1479A0E94F61F7A
:102AA0000E940A110E94721F0E94FC0340E061E034
:102AB00080E00E9448130E9485108257873130F4CD
:102AC000E82FF0E0E554FE4F808101C080E0909156
:102AD000620080FF02C0986001C0977F90936200FF
:102AE0009091620081FF02C0946001C09B7F90932F
:102AF00062009091620082FF02C0926001C09D7FDF
:102B00009093620083FF02C01D9A01C01D981C9A19
:102B1000A89AA998A99AAB9AAB98789480E008955E
:102B20000FB6F894A89581B5886181BD11BC0FBE20
:102B30000E943A15811130C09FE088E10FB6F894E9
:102B4000A89581BD0FBE91BDA8950E943B0F0E9424
:102B500040050E9463040E941D0480E00E9421063B
:102B6000813810F04FEF01C040E062E080E00E9449
:102B700048130E94DC1F882321F00E94201F0E941E
:102B8000731085B7837E85BF85B7806285BF8895C2
:102B900085B78F7D85BFD8CF80E090E00895CF9333
:102BA000DF930E94241191E090935D0710925E07DD
:102BB00091E590935F0792E19093600796E190937F
:102BC000610710926207109263071092640799E2FE
:102BD0009093650710926607109267071092680736
:102BE00091EC9093690710926A0710926B079CEC26
:102BF00090936C07E2EDF1E0ADE6B7E091919D9323
:102C000091E0EE3DF907D1F723E431E03093B407CA
:102C10002093B30793E39093B70727E031E0309315
:102C2000B2072093B1079CE39093B6072DE537E0F8
:102C30003093B0072093AF079CE19093B507282FFE
:102C400030E020573109359527952066C5EBD7E050
:102C5000EFEAF7E090E0A081B18139913550149608
:102C60003C93A081B18113963C9113974FEF430F92
:102C7000423020F419962C93199705C0323119F47B
:102C80001D962C931D979C93A081B18111961C9247
:102C9000A191B19115968C939F5F9330E1F6DF91EE
:102CA000CF910895CF93DF93E9E7F7E020E030E09C
:102CB00060ECAFEAB7E080E0CD91DD919B8191506F
:102CC000923038F44F81042E000C550B42175307F5
:102CD00019F08F5F833081F7A82FB0E0AA0FBB1FD8
:102CE000A155B84F0D90BC91A02D13969C911397B0
:102CF00090831C969C911C9795831D969C911D9783
:102D000097831182138214821282808766831396BE
:102D10008C911397813009F045C054968C9154974B
:102D2000807C91E009F490E091871E968D919C91B2
:102D30001F97982789279827968B858B50968D917A
:102D40009C915197982789279827908F878B5F961A
:102D50008C915F97828790968C91909783879196BC
:102D60008C919197848794968C919497858795966A
:102D70008C919597868796968C919697878797964C
:102D80008C919797808B98968C919897818B999638
:102D90008C919997828B9A968C919A97838B9B961C
:102DA0008C91848B2F5F3F4F7B962230310509F049
:102DB00080CFDF91CF910C940E20CF92DF92EF92D3
:102DC000FF920F931F93CF93DF931F92CDB7DEB780
:102DD000C82ED12C9BE1899F9001112489010758AD
:102DE000184FF801E080F1E0EF1231C6F82EF8013B
:102DF0008381843009F446C548F4813009F43CC32A
:102E000008F405C3823009F42FC417C6803109F4D1
:102E1000DEC0803221F0883009F00FC6DFC1F80132
:102E20009185618185854389992309F466C0062EC1
:102E3000000C770B082E000C990B042E000C550B80
:102E40004F5F5F4F841B950B86179707E4F0F901DE
:102E5000EE56F84F808180FF0CC09BE099838E7FF7
:102E6000808321E0AE014F5F5F4F60E88C2D0E94B0
:102E7000D90F8BE18C9DF0018D9DF00D1124E75849
:102E8000F84F80E183838BE18C9DF0018D9DF00DE7
:102E90001124DF01A758B84F14969C9114971396EC
:102EA0008C911397981761F011969C9111971D962C
:102EB0008C9189172CF0EE56F84F808181FF60C00D
:102EC0008BE18C9DF0018D9DF00D1124DF01A75841
:102ED000B84F11962C911197022E000C330B54967B
:102EE0008C915497082E000C990B01961D964C91CD
:102EF000840F911D47FD9A955DC070E090E050E011
:102F00004F5F5F4F841B950B86179707E4F0F9011D
:102F1000EE56F84F808180FF0CC09BE099838E7F36
:102F2000808321E0AE014F5F5F4F60E88C2D0E94EF
:102F3000D90F8BE18C9DF0018D9DF00D1124E75888
:102F4000F84F80E183838BE18C9DF0018D9DF00D26
:102F50001124DF01A758B84F14969C91149713962B
:102F60008C911397981781F011969C9111971D964B
:102F70008C91891748F0EE56F84F808181FD04C08E
:102F80009AE09983826026C58BE18C9DF0018D9D2E
:102F9000F00D1124DF01A758B84F11962C9111970D
:102FA00030E054968C91549790E001961D964C9188
:102FB000840F911D281739070CF43FC5EE56F84FC2
:102FC000808181FF3AC59AE099838D7F2DC5F801F4
:102FD000418581819585442309F47EC089179CF041
:102FE0008BE08983F901EE56F84F80818160808300
:102FF00021E0AE014F5F5F4F60E08C2D0E94D90F42
:1030000080E2F8012EC0082E000C990BF8014685CD
:10301000042E000C550B6389062E000C770B6F5F96
:103020007F4F461B570B48175907E4F0F901EE563E
:10303000F84F808182FF0CC099E099838B7F808359
:1030400021E0AE014F5F5F4F60E88C2D0E94D90FE9
:103050008BE18C9DF0018D9DF00D1124E758F84F08
:1030600088E083838BE18C9DF0018D9DF00D112410
:10307000DF01A758B84F14969C91149713968C9122
:103080001397981761F011969C9111971E968C9149
:1030900089172CF0EE56F84F808183FF78C08BE1C2
:1030A0008C9DF0018D9DF00D1124DF01A758B84FC4
:1030B00011962C911197022E000C330B54968C9183
:1030C0005497082E000C990B01961E964C91840F74
:1030D000911D47FD9A9575C0891798F08BE08983FB
:1030E000F901EE56F84F80818160808321E0AE01C6
:1030F0004F5F5F4F60E08C2D0E94D90F80E2F80196
:1031000028C090E0F801468550E0638970E06F5F69
:103110007F4F461B570B48175907E4F0F901EE564D
:10312000F84F808182FF0CC099E099838B7F808368
:1031300021E0AE014F5F5F4F60E88C2D0E94D90FF8
:103140008BE18C9DF0018D9DF00D1124E758F84F17
:1031500088E083838BE18C9DF0018D9DF00D11241F
:10316000DF01A758B84F14969C91149713968C9131
:103170001397981781F011969C9111971E968C9138
:10318000891748F0EE56F84F808183FD04C098E01F
:10319000998388601FC48BE18C9DF0018D9DF00D9B
:1031A0001124DF01A758B84F11962C91119730E0E8
:1031B00054968C91549790E001961E964C91840FF2
:1031C000911D281739070CF438C4EE56F84F80814A
:1031D00083FF33C498E09983877F26C4F801418533
:1031E00081819685442309F487C08917A4F089E07A
:1031F0008983F901EE56F84F80818460808321E055
:10320000AE014F5F5F4F60E08C2D0E94D90F80E1CF
:10321000F801838337C0082E000C990BF80147850D
:10322000042E000C550B6389062E000C770B6F5F84
:103230007F4F461B570B4817590724F1F901EE56EB
:10324000F84F808184FF15C087E089838BE18C9DD6
:10325000F0018D9DF00D1124EE56F84F80818F7E88
:10326000808321E0AE014F5F5F4F60E88C2D0E94AC
:10327000D90F8BE18C9DF0018D9DF00D1124E75845
:10328000F84F13828BE18C9DF0018D9DF00D112480
:10329000DF01A758B84F14969C91149713968C9100
:1032A0001397981761F011969C9111971F968C9126
:1032B00089172CF0EE56F84F808185FF81C08BE195
:1032C0008C9DF0018D9DF00D1124DF01A758B84FA2
:1032D00011962C911197022E000C330B54968C9161
:1032E0005497082E000C990B01961F964C91840F51
:1032F000911D47FD9A957EC08917A0F089E08983CA
:10330000F901EE56F84F80818460808321E0AE01A0
:103310004F5F5F4F60E08C2D0E94D90F80E1F80174
:10332000838331C090E0F801478550E0638970E005
:103330006F5F7F4F461B570B4817590724F1F90160
:10334000EE56F84F808184FF15C087E089838BE1BA
:103350008C9DF0018D9DF00D1124EE56F84F80816B
:103360008F7E808321E0AE014F5F5F4F60E88C2D40
:103370000E94D90F8BE18C9DF0018D9DF00D1124E1
:10338000E758F84F13828BE18C9DF0018D9DF00D75
:103390001124DF01A758B84F14969C9114971396E7
:1033A0008C911397981781F011969C9111971F9605
:1033B0008C91891748F0EE56F84F808185FD04C046
:1033C00096E09983806206C38BE18C9DF0018D9D10
:1033D000F00D1124DF01A758B84F11962C911197C9
:1033E00030E054968C91549790E001961F964C9142
:1033F000840F911D281739070CF41FC3EE56F84FA0
:10340000808185FF1AC396E099838F7D0DC3F801F3
:10341000418581819785442341F0891744F4F8015F
:10342000928998170CF409C31BC08917A0F087E094
:103430008983F901EE56F84F80818061808321E015
:10344000AE014F5F5F4F60E08F2D0E94D90F88E083
:10345000F8018383F2C2F8019289981708F4EDC24B
:10346000198221E0AE014F5F5F4F60E08F2D0E9417
:10347000D90FF801E382E1C2F801518541819189B8
:10348000552309F472C09417A4F083E08983F901ED
:10349000EE56F84F81818160818321E0AE014F5F5C
:1034A0005F4F60E08C2D0E94D90F82E0F80183838A
:1034B0002DC0042E000C550BF8016389062E000C5C
:1034C000770B6F5F7F4F9289690F711D97FD7A951A
:1034D00046175707DCF0F901EE56F84F908194FF3C
:1034E0000CC0898381818B7F818321E0AE014F5F96
:1034F0005F4F60E88C2D0E94D90F8BE18C9DF0010D
:103500008D9DF00D1124E758F84F13828BE18C9DAF
:10351000F0018D9DF00D1124DF01A758B84F1496CE
:103520009C91149713968C911397981741F01196CC
:103530009C91119752968C9198170CF06BC02BE1CF
:103540002C9DC0012D9D900D1124FC01E758F84FD2
:103550006181062E000C770B2289022E000C330BA2
:103560004489042E000C550B6AC09417A0F083E028
:103570008983F901EE56F84F81818160818321E0D2
:10358000AE014F5F5F4F60E08C2D0E94D90F82E04B
:10359000F801838327C050E0F801638970E06F5F12
:1035A0007F4F9289690F711D46175707DCF0F901AB
:1035B000EE56F84F908194FF0CC0898381818B7FF8
:1035C000818321E0AE014F5F5F4F60E88C2D0E9448
:1035D000D90F8BE18C9DF0018D9DF00D1124E758E2
:1035E000F84F13828BE18C9DF0018D9DF00D11241D
:1035F000DF01A758B84F14969C91149713968C919D
:103600001397981769F011969C91119752968C9187
:10361000981730F01982EE56F84F8181886020C1EA
:103620002BE12C9DC0012D9D900D1124FC01E7582C
:10363000F84F618170E0228930E0448950E04F5FAB
:103640005F4F241B350B261737070CF4F6C1FC011E
:10365000ED56F84F208123FFF0C11982FC01EE5690
:10366000F84F8181877F96C0F801418581819089DB
:10367000442309F491C098179CF085E08983F901EF
:10368000EE56F84F80818064808321E0AE014F5F69
:103690005F4F60E08C2D0E94D90F84E0F80136C0A6
:1036A000082E000C990BF8014389042E000C550BD1
:1036B0004F5F5F4F6189460F511D67FD5A95841713
:1036C00095072CF1F901EE56F84F808182FF15C065
:1036D00083E089838BE18C9DF0018D9DF00D112499
:1036E000EE56F84F81818E7F818321E0AE014F5FDE
:1036F0005F4F60E88C2D0E94D90F8BE18C9DF0010B
:103700008D9DF00D1124E758F84F81E083838BE104
:103710008C9DF0018D9DF00D1124DF01A758B84F4D
:1037200014969C91149713968C911397981741F0C7
:1037300011969C91119751968C9198170CF08AC014
:103740002BE12C9DC0012D9D900D1124FC01E7580B
:10375000F84F6181062E000C770B2189022E000C98
:10376000330B4489042E000C550B4F5F5F4F241B15
:10377000350B261737070CF460C1FC01ED56F84FE6
:10378000208121FF5AC122E02983FC01EE56F84F27
:1037900081818D7F818349C1981798F085E0898365
:1037A000F901EE56F84F80818064808321E0AE01FC
:1037B0004F5F5F4F60E08C2D0E94D90F84E0F801CD
:1037C00030C090E0F801438950E04F5F5F4F61895E
:1037D000460F511D841795072CF1F901EE56F84F4D
:1037E000808182FF15C083E089838BE18C9DF0018D
:1037F0008D9DF00D1124EE56F84F81818E7F8183CF
:1038000021E0AE014F5F5F4F60E88C2D0E94D90F21
:103810008BE18C9DF0018D9DF00D1124E758F84F40
:1038200081E083838BE18C9DF0018D9DF00D11244F
:10383000DF01A758B84F14969C91149713968C915A
:103840001397981779F011969C91119751968C9136
:10385000981740F082E08983EE56F84F81818260AC
:103860008183B9C02BE12C9DC0012D9D900D1124A9
:10387000FC01E758F84F618170E0218930E044890C
:1038800050E073CFF8019185418183896089992344
:1038900009F45EC0042E000C550B082E000C990B89
:1038A0000196860F911D67FD9A9548175907E4F018
:1038B000F901EE56F84F808180FF0CC095E09983A6
:1038C0008F7B808321E0AE014F5F5F4F60E88C2DDE
:1038D0000E94D90F8BE18C9DF0018D9DF00D11247C
:1038E000E758F84F82E083838BE18C9DF0018D9D3A
:1038F000F00D1124DF01A758B84F14969C9114972E
:1039000013968C911397981741F011969C911197EB
:1039100050968C9198170CF057C08BE18C9DF0015C
:103920008D9DF00D1124DF01A758B84F11964C91D1
:103930001197042E000C550B51968C915197082E1F
:10394000000C990B54962C91022E000C330B5DC089
:1039500050E090E00196860F911D48175907E4F05A
:10396000F901EE56F84F808180FF0CC095E09983F5
:103970008F7B808321E0AE014F5F5F4F60E88C2D2D
:103980000E94D90F8BE18C9DF0018D9DF00D1124CB
:10399000E758F84F82E083838BE18C9DF0018D9D89
:1039A000F00D1124DF01A758B84F14969C9114977D
:1039B00013968C9113979817A1F011969C911197DB
:1039C00050968C91981768F084E08983EE56F84FF2
:1039D00080818068808321E0AE014F5F5F4F60E0AF
:1039E00029C08BE18C9DF0018D9DF00D1124DF012C
:1039F000A758B84F11964C91119750E051968C9161
:103A0000519790E054962C9130E02F5F3F4F821BEE
:103A1000930B841795078CF0EE56F84F808187FF43
:103A20000CC094E099838F77808321E0AE014F5FD3
:103A30005F4F60E88F2D0E94D90F8BE18C9DF001C4
:103A40008D9DF00D1124E758F84F838184830F90EA
:103A5000DF91CF911F910F91FF90EF90DF90CF906A
:103A60000895611102C022E001C023E0FC0120831F
:103A700021E0218382E00895CF93DF93F901DC01F7
:103A80008D919C9184309105E8F54D33D8F56134E2
:103A9000C8F58330910561F0A42FB0E0A60FB11DE9
:103AA000EC01CB54D84F288130E02A173B0754F162
:103AB0009C012F5F3F4F2330310528F421E0280F70
:103AC0002083118206C02FEF20832183833091054C
:103AD000D9F0262F30E0DF011296880F991FFC01E4
:103AE000E155F84F822F861B841748F4C081D1819D
:103AF000C20FD31F88818D932F5F3F4FF3CF82E09A
:103B0000840F03C08FEF01C082E0DF91CF91089551
:103B1000CF93DF93FB01282F30E0233031050CF0E9
:103B200073C0823008F072C08BE1829FD001839F06
:103B3000B00D1124A758B84F1896CC911897D0E023
:103B4000CC0FDD1FC155D84F0990D881C02D8B8176
:103B5000813009F051C08FE380831896CC9118977B
:103B6000D0E0CC0FDD1FC155D84F0990D881C02DB2
:103B700089A581831896CC911897D0E0CC0FDD1FD2
:103B8000C155D84F0990D881C02D88A58283189639
:103B9000CC911897D0E0CC0FDD1FC155D84F0990BC
:103BA000D881C02D8FA183831896CC911897D0E02F
:103BB000CC0FDD1FC155D84F0990D881C02D8EA1E3
:103BC00084831896CC911897D0E0CC0FDD1FC15597
:103BD000D84F0990D881C02D8DA185831896AC91BE
:103BE000B0E0AA0FBB1FA155B84F0D90BC91A02DFE
:103BF00094968C9186830AC010821182128213825D
:103C000014821582168202C08FEF01C087E0DF9117
:103C1000CF910895AF92CF92EF920F93E82FF0E0FB
:103C2000E330F1050CF08EC0823008F089C08BE1E2
:103C30008E9FD0018F9FB00D1124A758B84F1896B2
:103C4000AC91B0E0AA0FBB1FA155B84F0D90BC912D
:103C5000A02D13968C911397813009F071C060FFED
:103C600002C099964C9361FF14C08BE18E9FD001E6
:103C70008F9FB00D1124A758B84F1896AC91B0E0A3
:103C8000AA0FBB1FA155B84F0D90BC91A02D9896BF
:103C90002C9362FF14C08BE18E9FD0018F9FB00DDB
:103CA0001124A758B84F1896AC91B0E0AA0FBB1FCB
:103CB000A155B84F0D90BC91A02D97960C9363FF22
:103CC00014C08BE18E9FD0018F9FB00D1124A75897
:103CD000B84F1896AC91B0E0AA0FBB1FA155B84FD2
:103CE0000D90BC91A02D9696EC9264FF14C08BE1D0
:103CF0008E9FD0018F9FB00D1124A758B84F1896F2
:103D0000AC91B0E0AA0FBB1FA155B84F0D90BC916C
:103D1000A02D9596CC9265FF13C02BE12E9FC0017C
:103D20002F9F900D1124FC01E758F84FE085F0E03B
:103D3000EE0FFF1FE155F84F0190F081E02DA4A296
:103D400080E001C08FEF0F91EF90CF90AF9008957A
:103D5000FB0190E08330910564F52BE1289FD001B1
:103D6000299FB00D1124A758B84F15962C9115977F
:103D7000223F11F4108203C011962C9120832BE175
:103D8000289FD001299FB00D1124A758B84F16962F
:103D90008C911697818315968C911597823F19F413
:103DA00011968C9102C013968C918283138284E0C9
:103DB00008958FEF0895811109C080915D07FB017F
:103DC000808380915E07818382E008958FEF08955C
:103DD0002BE1829FC0011124FC01E758F84F618359
:103DE00008952BE1829FC0011124FC01E758F84F90
:103DF000818108952BE1829FC0011124FC01E758C5
:103E0000F84F81E0828308952BE1829FC001112445
:103E1000FC01E758F84F8281128208952BE1829FBE
:103E2000C0011124FC01E758F84F858108952BE16A
:103E3000829FC0011124FC01E758F84F8781089543
:103E40000E940F2080E00E942106809395078091B8
:103E50007F07803C41F480917E078150823018F4C6
:103E600080E00E94DD1680919A07803C41F48091A9
:103E700099078150823018F481E00C94DD16089582
:103E8000039666E170E00E94D2208CE0869F90014C
:103E9000879F300D112480E090E08217930719F07E
:103EA00000000196FACF0895039666E170E00E9443
:103EB000D2208CE0869FA001879F500D112428EE10
:103EC00033E080E090E08417950719F00000019638
:103ED000FACF21503109A9F7089593B7987F892B1C
:103EE00083BF08951092B9071092B8071092A302E9
:103EF0001092A2021092A1021092A00210929F02B0
:103F000083B7886083BF83E00E946D1F12BE8CE878
:103F100081BF87B7826087BF08951F920F920FB647
:103F20000F9211240BB60F922F933F934F935F93F1
:103F30006F937F938F939F93AF93BF93EF93FF9371
:103F40008091A1029091A20201969093A202809387
:103F5000A10220919F023091A0022F5F3F4F30932A
:103F6000A00220939F02099734F01092A2021092AF
:103F7000A1020E94FB1480919F029091A0028436BE
:103F800091053CF081E08093A3021092A002109270
:103F90009F02FF91EF91BF91AF919F918F917F9180
:103FA0006F915F914F913F912F910F900BBE0F90AA
:103FB0000FBE0F901F9018958091A3021092A3023C
:103FC00008959C0190E0615030F0F901E60FF11D79
:103FD0008081980FF8CF892F81950895CF93C42FB2
:103FE0000E94E11FC81B8C2FCF91089561E080E0F3
:103FF0000E94E90661E081E00E94E90661E082E05A
:104000000E94E90661E083E00E94E90661E084E045
:104010000C94E90681E0089581E0089508950895DB
:1040200089B381700895CF92DF92EF92FF920F9340
:104030001F93CF93DF93DA01F801E7011882108212
:10404000118290E69283813091F511969C9199307E
:1040500010F089EC9AC0E8016A01182F0E94102024
:10406000811104C092E0F701908393C093B3892F2C
:10407000807295FD03C0F70110838BC0F60160814B
:1040800070E000E010E020E041E081E60E944A0B91
:104090008E010D5F1F4FF601218140E060E070E06E
:1040A00081E60E94E20BF60181818D5F72C0833050
:1040B00009F06AC08C9180FF08C011968C9111970D
:1040C00080FF02C0A89A01C0A8988C9181FF08C007
:1040D00011968C91119781FF02C0A99A01C0A998ED
:1040E0008C9182FF08C011968C91119782FF02C0BB
:1040F000AA9A01C0AA988C9183FF08C011968C914E
:10410000119783FF02C0AB9A01C0AB988C9186FFD8
:1041100008C011968C91119786FF02C01C9A01C0AD
:104120001C988C9187FF07C011968C9187FF02C065
:104130001F9A01C01F981382989B02C081E083835D
:10414000999B03C08381826083839A9B03C0838190
:10415000846083839B9B03C08381886083839C9B53
:1041600003C08381806183839D9B03C083818062C0
:1041700083830C9B03C08381806483830F9B08C06F
:1041800083818068838304C081EC888380E001C0E0
:1041900084E0DF91CF911F910F91FF90EF90DF901E
:1041A000CF900895AA1BBB1B51E107C0AA1FBB1FDC
:1041B000A617B70710F0A61BB70B881F991F5A95B3
:1041C000A9F780959095BC01CD010895EE0FFF1FD2
:1041D0000024001C0BBE0790F691E02D09940F936C
:1041E0001F93CF93DF938230910510F482E090E02B
:1041F000E091BE07F091BF0720E030E0A0E0B0E022
:10420000309719F140815181028113814817590774
:10421000C8F08417950769F4109731F012960C9343
:10422000129713961C9327C00093BE071093BF07E5
:1042300022C02115310519F04217530718F49A01CD
:10424000BD01EF01DF01F801DBCF21153105F9F0E8
:10425000281B390B2430310580F48A819B8161153C
:10426000710521F0FB019383828304C09093BF0703
:104270008093BE07FE01329644C0FE01E20FF31F99
:104280008193919322503109398328833AC0209138
:10429000BC073091BD07232B41F4209102013091DE
:1042A00003013093BD072093BC072091000130919A
:1042B00001012115310541F42DB73EB740910401AC
:1042C00050910501241B350BE091BC07F091BD070F
:1042D000E217F307A0F42E1B3F0B2817390778F0DD
:1042E000AC014E5F5F4F2417350748F04E0F5F1F3C
:1042F0005093BD074093BC078193919302C0E0E0C7
:10430000F0E0CF01DF91CF911F910F910895CF93EE
:10431000DF93009709F481C0FC0132971382128267
:10432000A091BE07B091BF07109781F42081318121
:10433000820F931F2091BC073091BD0728173907C2
:1043400051F5F093BD07E093BC0767C0ED0120E095
:1043500030E0CE17DF0740F44A815B819E014115B2
:104360005105F1F0EA01F5CFD383C2834081518139
:10437000840F951FC817D90759F488819981840F34
:10438000951F0296918380838A819B819383828388
:104390002115310529F4F093BF07E093BE073DC016
:1043A000E901FB83EA8349915991C40FD51FEC17AA
:1043B000FD0761F480819181840F951F0296E901C8
:1043C00099838883828193819B838A83E0E0F0E0F4
:1043D00012968D919C911397009719F0FD01DC01C5
:1043E000F7CF8D919C9111979D012E5F3F4F820FCA
:1043F000931F2091BC073091BD072817390769F436
:10440000309729F41092BF071092BE0702C01382A2
:104410001282B093BD07A093BC07DF91CF9108959E
:04442000F894FFCF3E
:104424000000C0072000FF0300510137000000C155
:104434000003C1F26F070000000700C00000000085
:104444000000000000000000000000000000000068
:10445400000000000000CC414D4320484F545F53FE
:104464005741500000510100000001C1007FFC02CF
:1044740001FF7FFF7F0000000400004D02400100A7
:10448400DE079AB481FF00F5CEB481674D060600BD
:104494000000C3313256495032495F414D435F41B8
:1044A400444336345F5632003030303030303030B0
:1044B400310044554E455F414D4300436F7265469C
:1044C40052550044554E455F414D435F4144433688
:1044D40034004345524E204D4D4300010002000379
:1044E400000400050006000700080009000A000B8C
:1044F400000C44554E455F5444455F414D43000014
:00000001FF
